:200000000C948A000C949C000C949C000C949C000C949C000C949C000C949C000C949C0012
:200020000C949C000C949C000C949C000C949C000C949C000C949C000C949C000C949C00E0
:200040000C949C000C949C000C94B6000C949C000C949C000C949C000C949C000C949C00A6
:200060000C949C000C949C000C949C000C949C000C949C000C949C000C949C000C949C00A0
:200080000C949C000C949C000C949C00A701AA019D01A101C101C101AE01B201B801BC01BD
:2000A000000000010200090A00000000040308070000000000000000000000000000000014
:2000C000010204081020408001020408102040800102040810204080010204081020408024
:2000E0000202020202020202040404040404040403030303030303030101010101010101B0
:2001000000002200250028002B0000002100240027002A0011241FBECFEFD0E4DEBFCDBF02
:2001200021E0A0E0B1E001C01D92A930B207E1F70E9432020C9448020C94000061E08DE0C5
:200140000C94C20161E08DE00E94FB0168EE73E080E090E00E94230160E08DE00E94FB0166
:2001600068EE73E080E090E00C9423011F920F920FB60F9211242F933F938F939F93AF932B
:20018000BF938091010190910201A0910301B09104013091000123E0230F2D3720F4019655
:2001A000A11DB11D05C026E8230F0296A11DB11D209300018093010190930201A093030164
:2001C000B09304018091050190910601A0910701B09108010196A11DB11D809305019093B6
:2001E0000601A0930701B0930801BF91AF919F918F913F912F910F900FBE0F901F9018959A
:200200003FB7F8948091050190910601A0910701B091080126B5A89B05C02F3F19F00196A9
:20022000A11DB11D3FBF6627782F892F9A2F620F711D811D911D42E0660F771F881F991FA8
:200240004A95D1F70895CF92DF92EF92FF92CF93DF936B017C010E940001EB01C114D10480
:20026000E104F10489F00E9441020E9400016C1B7D0B683E734090F381E0C81AD108E108B3
:20028000F108C851DC4FEACFDF91CF91FF90EF90DF90CF900895789484B5826084BD84B57E
:2002A000816084BD85B5826085BD85B5816085BDEEE6F0E0808181608083E1E8F0E01082AD
:2002C000808182608083808181608083E0E8F0E0808181608083E1EBF0E080818460808352
:2002E000E0EBF0E0808181608083E1E9F0E0808182608083808181608083E0E9F0E080817F
:2003000081608083EAE7F0E0808184608083808182608083808181608083808180688083B9
:200320001092C100089590E0FC013197EA30F10540F5EA5BFF4F0C944202809180008F7735
:2003400003C0809180008F7D80938000089584B58F7702C084B58F7D84BD08958091B00028
:200360008F7703C08091B0008F7D8093B0000895809190008F7703C0809190008F7D80935D
:2003800090000895CF93DF9390E0FC01E054FF4F2491FC01E052FF4F8491882349F190E0D1
:2003A000880F991FFC01E65FFE4FA591B49180509F4FFC01C591D4919FB7611108C0F89452
:2003C0008C91209582238C93888182230AC0623051F4F8948C91322F309583238C9388819B
:2003E000822B888304C0F8948C91822B8C939FBFDF91CF9108950F931F93CF93DF931F9268
:20040000CDB7DEB7282F30E0F901E056FF4F8491F901E054FF4F1491F901E052FF4F049199
:200420000023C9F0882321F069830E9493016981E02FF0E0EE0FFF1FE050FF4FA591B49125
:200440009FB7F8948C91611103C01095812301C0812B8C939FBF0F90DF91CF911F910F9176
:20046000089508950E944B010E9431020E949E00C0E0D0E00E94A2002097E1F30E9400007E
:20048000F9CF0895EE0FFF1F0590F491E02D0994F894FFCFFFFFFFFFFFFFFFFFFFFFFFFFCA
:2004A000FFFFFFFFFFFFFFFFFFFFFFFFFFFFFFFFFFFFFFFFFFFFFFFFFFFFFFFFFFFFFFFF5C
:2004C000FFFFFFFFFFFFFFFFFFFFFFFFFFFFFFFFFFFFFFFFFFFFFFFFFFFFFFFFFFFFFFFF3C
:2004E000FFFFFFFFFFFFFFFFFFFFFFFFFFFFFFFFFFFFFFFFFFFFFFFFFFFFFFFFFFFFFFFF1C
:2005000000226349497F360000181814167F7F1000276745457D3900003E7F49497B3200DD
:20052000000303797D07030000367F49497F360000266F49497F3E0000000024240000008D
:20054000000080E46400000000081C3663414100001414141414140000414163361C0800DD
:2005600000020351590F0600003E7F414D4F2E00007C7E0B0B7E7C00007F7F49497F3600A0
:20058000003E7F4141632200007F7F41633E1C00007F7F4949414100007F7F090901010077
:2005A000003E7F41497B3A00007F7F08087F7F000000417F7F410000002060417F3F010033
:2005C000007F7F1C36634100007F7F4040404000007F7F060C067F7F007F7F0E1C7F7F00EF
:2005E000003E7F41417F3E00007F7F09090F0600001E3F21617F5E00007F7F19396F460019
:2006000000266F49497B32000001017F7F010100003F7F40407F3F00001F3F60603F1F008C
:20062000007F7F3018307F7F0063771C1C77630000070F78780F0700006171594D4743003C
:2006400000007F7F4141000040687C5E49492200000041417F7F00001818181818181818A4
:2006600000185C7E7F7E5C18000000FFFF00000000207454547C7800007F7F44447C3800AF
:2006800000387C44446C280000387C44447F7F0000387C54545C580000087E7F090302002D
:2006A0000098BCA4A4FC7C00007F7F04047C78000000007D7D0000000040C08080FD7D00B8
:2006C000007F7F30386C44000000417F7F400000007C7C181C187C7C007C7C04047C780055
:2006E00000387C44447C380000FCFC24243C180000183C2424FCFC00007C7C04040C0800CE
:2007000000485C545474200004043F7F44642000003C7C40407C3C00001C3C60603C1C000B
:20072000001C7C3018307C1C00446C38386C4400009CBCA0A0FC7C00004464745C4C440029
:2007400018181818181818180C0C0C0C0C0C0C0C06060606060606063030303030303030C9
:200760000000FFFF0000000000000000FFFF0000181838F0E0000000000000070F1C1818E3
:2007800018181C0F07000000FFFFC0C0C0C0C0C003070E1C3870E0C0C0E070381C0E070381
:2007A000FFFF030303030303030303030303FFFF003C7E7E7E7E3C006060606060606060A9
:2007C000000E1F3F7E3F1F0E00FFFF0000000000000000E0F0381818C3E77E3C3C7EE7C3C5
:2007E000003C7E66667E3C00000C4C73734C0C000000000000FFFF0000081C3E7F3E1C08E2
:20080000181818FFFF1818183333CCCC00000000000000FFFF0000000010787808787C044E
:200820000103070F1F3F7FFF0000000000000000FFFFFFFF00000000F0F0F0F0F0F0F0F046
:2008400001010101010101018080808080808080FFFF0000000000003333CCCC3333CCCC96
:20086000000000000000FFFF3030C0C03030C0C0FF7F3F1F0F070301000000000000FFFFC6
:20088000000000FFFF18181800000000F0F0F0F00000001F1F181818181818F8F800000094
:2008A000C0C0C0C0C0C0C0C0000000F8F81818181818181F1F181818181818F8F8181818B2
:2008C000181818FFFF000000FFFF000000000000FFFFFF00000000000000000000FFFFFFDA
:2008E00003030303030303030707070707070707E0E0E0E0E0E0E0E0C0C0C0C0C0C0FFFF2A
:20090000F0F0F0F000000000000000000F0F0F0F1818181F1F0000000F0F0F0F0000000019
:200920000F0F0F0FF0F0F0F01818181818181818181818FFFF1818183333CCCC000000006F
:20094000000000FFFF000000CCCC3333CCCC333366CC993366CC99330000000000000000A1
:20096000FFFFFFFF00000000F0F0F0F0F0F0F0F001010101010101018080808080808080F3
:20098000FFFF0000000000003333CCCC3333CCCC000000000000FFFF3030C0C03030C0C09F
:2009A0003399CC663399CC66000000000000FFFF000000FFFF18181800000000F0F0F0F037
:2009C0000000001F1F181818181818F8F8000000C0C0C0C0C0C0C0C0000000F8F818181821
:2009E0001818181F1F181818181818F8F8181818181818FFFF000000FFFF00000000000065
:200A0000FFFFFF00000000000000000000FFFFFF030303030303030307070707070707078C
:200A2000E0E0E0E0E0E0E0E000787830180C0603F0F0F0F000000000000000000F0F0F0F6D
:200A40001818181F1F0000000F0F0F0F000000000F0F0F0FF0F0F0F00000000000000000D8
:200A6000000000000000000000000000000000000000000000000000000000000000000076
:200A8000000000000000000000000000000000000000000000000000000000000000000056
:200AA000000000000000000000000000000000000000000000000000000000000000000036
:200AC000000000000000000000000000000000000000000000000000000000000000000016
:200AE0000000000000000000000000000000000000000000000000000000000000000000F6
:200B00000000000000000000000000000000000000000000000000000000000000000000D5
:200B20000000000000000000000000000000000000000000000000000000000000000000B5
:200B4000000000000000000000000000000000000000000000000000000000000000000095
:200B600000000000000000004500008200004000200001080006040001003108B70EFC112F
:200B8000A43411241FBECFEFD0E4DEBFCDBF12E0A0E0B1E0EAE3F1E700E00BBF02C0079025
:200BA0000D92AE35B107D9F72CE0AEE5B2E001C01D92A834B207E1F71BE0C2E8DBE000E0DD
:200BC00006C022970109FE010BBF0E948838CA37D10780E00807A9F70E94F80A0C946C3792
:200BE0000C940000DC011696ED91FC9117979F012F5F3F4F17963C932E931697608381E029
:200C000090E008950F931F93CF93DF93CDB7DEB72A970FB6F894DEBF0FBECDBF9B018A0157
:200C20004AE0BE016F5F7F4F07960E94DE2F882329F0CE0101960E944E378C01C8012A967C
:200C40000FB6F894DEBF0FBECDBFDF91CF911F910F9108951F93CF93DF93EC0110E0699133
:200C60004AE050E085E698E00E94CA0B133029F06EE285E698E00E94470B1F5F143079F70B
:200C8000DF91CF911F910895109261086FEE7BE785E698E00E9436236EE371E085E698E00A
:200CA0000E94450B60E187E998E00E94100D81110CC060E078EF85E698E00E94362369E529
:200CC00071E085E698E00C94520B60EE77E085E698E00E94362361E671E085E698E00E9443
:200CE000520B6FEE7BE785E698E00E94362381E080936108089561E082E00E94880A60E069
:200D000082E00E94C10A61E070E080E090E00E94E90961E082E00C94C10A0E947B066FEE81
:200D20007BE785E698E00E94362366E671E085E698E00E94450B41E06AE071E08CED95E057
:200D40000E94EB29811109C060E078EF85E698E00E94362369E571E063C060EE77E085E62B
:200D600098E00E94362361E671E085E698E00E94520B60E080E090E00E949F2581110CC0B2
:200D800060E078EF85E698E00E94362360E871E085E698E00E94520B6FEE7BE785E698E0B1
:200DA0000E9436236EE871E085E698E00E94450B6FEF7FEF85E698E00E94362380E59BE032
:200DC0000E942A066FEE7BE785E698E00E94362365E971E085E698E00E94450B6FEF7FEF64
:200DE00085E698E00E94362384E49BE00E942A066FEE7BE785E698E00E9436236DE971E01C
:200E000085E698E00E94450B6FEF7FEF85E698E00E9436238CE39BE00E942A0666EE71E0F2
:200E200085E698E00C94520B67E170E082E698E00E94321F6AE570E082E698E00C946B1FBE
:200E400061E085E10E94880A61E086E10E94880A61E083E00C94880A4F925F926F927F9221
:200E60008F929F92AF92BF92CF92DF92EF92FF921F93CF93DF930E942028909361028093A1
:200E800060020E94C92C90935F0280935E02009709F4D7C0109265021092640220EA32E00A
:200EA000309367022093660230936902209368029C0127593D4F79016FE178EF85E698E0E3
:200EC0000E943623F70186818F3381F540E050E06EEA71E0C7010E940206C82F4FEF5FEFF2
:200EE0006CE871E0C7010E9402066C01182F40E050E061EB71E0C7010E940206D82F8CEE47
:200F00008C0D873950F4DD24B60183E00E94FF08B60182E698E00E946B1F6C2F85E10E940A
:200F2000C10A6D2F86E10E94C10A03C0D0E0C0E01AE50E94BA0928EE33E040E050E00E94E4
:200F4000363849015A01CA01B90120E13EE040E050E00E94583829013A018CE3C82ED12C91
:200F6000E12CF12CC501B401A70196010E945838B62ECA01B901A70196010E945838362F1C
:200F80002AE08B2D622F0E941638D82EC92E832F0E941638F82EE92EC2016AE070E00E9433
:200FA0002238E12FF0E0DD2319F046EA51E002C047EE51E0CC2319F026EA31E002C027EE75
:200FC00031E01F92CF921F92DF921F92EF921F92FF929F938F937F936F93FF93EF935F93EA
:200FE0004F933F932F9384EB90E09F938F9382E692E09F938F930E94EC282DB73EB72A5E03
:201000003F4F0FB6F8943EBF0FBE2DBF80916802909169022091660230916702821B930BB6
:20102000DF91CF911F91FF90EF90DF90CF90BF90AF909F908F907F906F905F904F900C94FC
:201040009F2BDF91CF911F91FF90EF90DF90CF90BF90AF909F908F907F906F905F904F90B2
:2010600008952EE04CE06FE085E698E00E94503082E698E00E94981E86E498E00E948F0CEE
:20108000109265021092640281EE91E09093630280936202089560E070E085E698E00E94AE
:2010A0001F3040E050E060E070E085E698E00E942A2360EE7FEF85E698E00E94362362E053
:2010C00085E698E00E94302364EB71E085E698E00E94520B61E085E698E00C94302385E634
:2010E00098E00E94BD3263E085E698E00E94F9330C944B080F931F93CF93DF93CDB7DEB7BF
:201100006B970FB6F894DEBF0FBECDBF80916108882309F45DC021E044ED51E067E978E03C
:20112000CE0101960E94290E8B819C8190934908809348088D819E81AF81B88580934A0871
:2011400090934B08A0934C08B0934D0889859A85AB85BC8580934E0890934F08A0935008EE
:20116000B09351088DE0FE013D96A2E5B8E001900D928A95E1F78A8D9B8D90936008809371
:201180005F0886E498E00E94030D8823D9F086E498E00E94C20C892B81F0E0916508F0910A
:2011A00066080081118186E498E00E94210C682F85E698E0F8010995EACF86E498E00E94AF
:2011C000F10C06C066EC71E085E698E00E94520B6B960FB6F894DEBF0FBECDBFDF91CF91AF
:2011E0001F910F9108950E946F080E9444060E948D060E9414070E9420070C947A081F936E
:20120000CF93DF93182FEB0161E00E94880A209711F460E004C0CF3FD10539F461E0812F90
:20122000DF91CF911F910C94C10AE12FF0E0EC51FD4F449150E0FA013197EA30F10508F08A
:2012400046C0EA5BFF4F0C94773884B5806884BDC7BD42C084B5806284BDC8BD3DC08091CF
:201260008000806880938000D0938900C093880033C080918000806280938000D0938B00C5
:20128000C0938A0029C08091B00080688093B000C093B30021C08091B00080628093B000CF
:2012A000C093B40019C080919000806880939000D0939900C09398000FC0809190008062E9
:2012C00080939000D0939B00C0939A0005C0C038D1050CF0A3CF9DCFDF91CF911F910895F6
:2012E0001F920F920FB60F9211242F933F938F939F93AF93BF9380918F0890919008A091F3
:201300009108B091920830918E0823E0230F2D3720F40196A11DB11D05C026E8230F029695
:20132000A11DB11D20938E0880938F0890939008A0939108B0939208809193089091940861
:20134000A0919508B09196080196A11DB11D8093930890939408A0939508B0939608BF914F
:20136000AF919F918F913F912F910F900FBE0F901F9018952FB7F89460918F087091900853
:2013800080919108909192082FBF08953FB7F8948091930890919408A0919508B0919608C5
:2013A00026B5A89B05C02F3F19F00196A11DB11D3FBF6627782F892F9A2F620F711D811D60
:2013C000911D42E0660F771F881F991F4A95D1F70895CF92DF92EF92FF92CF93DF936B016B
:2013E0007C010E94C609EB01C114D104E104F10489F00E9437340E94C6096C1B7D0B683EE3
:20140000734090F381E0C81AD108E108F108C851DC4FEACFDF91CF91FF90EF90DF90CF90EF
:201420000895789484B5826084BD84B5816084BD85B5826085BD85B5816085BDEEE6F0E0ED
:20144000808181608083E1E8F0E01082808182608083808181608083E0E8F0E08081816037
:201460008083E1EBF0E0808184608083E0EBF0E0808181608083E1E9F0E0808182608083E5
:20148000808181608083E0E9F0E0808181608083EAE7F0E08081846080838081826080837A
:2014A0008081816080838081806880831092C100089590E0FC013197EA30F10540F5E05BA6
:2014C000FF4F0C947738809180008F7703C0809180008F7D80938000089584B58F7702C047
:2014E00084B58F7D84BD08958091B0008F7703C08091B0008F7D8093B00008958091900071
:201500008F7703C0809190008F7D809390000895CF93DF9390E0FC01EC5FFC4F2491FC018C
:20152000EC5DFC4F8491882349F190E0880F991FFC01E25BFC4FA591B4918C5B9C4FFC018F
:20154000C591D4919FB7611108C0F8948C91209582238C93888182230AC0623051F4F89443
:201560008C91322F309583238C938881822B888304C0F8948C91822B8C939FBFDF91CF913B
:2015800008950F931F93CF93DF931F92CDB7DEB7282F30E0F901EC51FD4F8491F901EC5F78
:2015A000FC4F1491F901EC5DFC4F04910023C9F0882321F069830E94590A6981E02FF0E0C6
:2015C000EE0FFF1FEC5BFC4FA591B4919FB7F8948C91611103C01095812301C0812B8C93DA
:2015E0009FBF0F90DF91CF911F910F91089508950E94110A0E94F70A0E94F308C4E1D5E33A
:201600000E942C072097E1F30E941435F9CFCF92DF92EF92FF920F931F93CF93DF936C013E
:201620007A01EB01E60EF71E00E010E0CE15DF0561F06991D601ED91FC910190F081E02D67
:20164000C6010995080F191FF1CFC801DF91CF911F910F91FF90EF90DF90CF90089561153E
:20166000710581F0DB010D900020E9F7AD0141505109461B570BDC01ED91FC910280F381D0
:20168000E02D099480E090E008950C942F0BDC01ED91FC910190F081E02D099465EE71E021
:2016A0000C942F0B0F931F93CF93DF93EC010E942F0B8C01CE010E944E0B800F911FDF9159
:2016C000CF911F910F9108958F929F92AF92BF92CF92DF92EF92FF920F931F93CF93DF93CD
:2016E000CDB7DEB7A1970FB6F894DEBF0FBECDBF7C01C42EE52FCB01D22E19A221E02D1505
:2017000010F02AE0D22E8E010F5D1F4F8D2C912CA12CB12C6C2D7E2FA50194010E943638A5
:201720008C2DD29E80191124015011098A3014F4805D01C0895CF801808321153105410554
:20174000510521F0C22EE32FCA01E4CFB801C7010E942F0BA1960FB6F894DEBF0FBECDBFC7
:20176000DF91CF911F910F91FF90EF90DF90CF90BF90AF909F908F9008952115310541F453
:20178000DC01ED91FC910190F081E02D642F09940C94640B9A01462F50E060E070E00C94A3
:2017A000BD0BCF93DF931F92CDB7DEB76983DC01ED91FC910280F381E02D41E050E0BE01DC
:2017C0006F5F7F4F09950F90DF91CF910895CF93DF93EC01898D9A8D009759F0FC01138253
:2017E00012820E947D17E98DFA8D22813381232B31F081E090E09B838A8380E090E0DF9120
:20180000CF910895FC01818D928D009711F00C941D150895CF93DF931F92CDB7DEB741E0DB
:2018200050E0BE016F5F7F4F0E942E13019719F4898190E002C08FEF9FEF0F90DF91CF91DE
:201840000895FC01818D928D009711F00C940A0C8FEF9FEF08950F931F93CF93DF938C0115
:20186000FC01818D928D0097B9F00E940A0CEC018F3FFFEF9F0799F0F801818D928DFC014B
:20188000428553856485758541505109610971090E948114CE0105C080E090E002C08FEF1C
:2018A0009FEFDF91CF911F910F910895CF92DF92EF92FF920F931F93CF93DF93EC017B0168
:2018C0006A011B821A8208EE13E020E030E00C831D832E833F838AEF91E0998388838DE14A
:2018E00090E00E9422369A8F898F009779F02DE1F701DC0101900D922A95E1F74CE050E037
:20190000B601CE010C960E94A637188EDF91CF911F910F91FF90EF90DF90CF900895FC01E4
:201920001382128248EE53E060E070E044835583668377838AEF91E091838083128E118EC3
:2019400014860895DC015996ED91FC915A97309729F0628573858485958508956FEF7FEF3D
:20196000CB010895DC015996ED91FC915A97309729F06389748985899689089560E070E013
:20198000CB010895CF92DF92EF92FF92CF93DF93EC01898D9A8D892BD9F0CE010E94B20C50
:2019A0006B017C01CE010E94A20CA7019601261B370B480B590BDA01C901811530E89307B9
:2019C000A105B10538F08FEF9FE7A0E0B0E002C080E090E0DF91CF91FF90EF90DF90CF9031
:2019E0000895CF93DF93EC01898D9A8D009741F00E946415898D9A8D0E94BA361A8E198E4B
:201A0000DF91CF910895DC015996ED91FC915A97309721F081E09581911101C080E00895E2
:201A20000F931F93CF93DF93EC01462F61E00E94F40F811102C080E01DC08E01045F1F4F45
:201A400041E0BE01C8010E94C41C882359F0B801CE018A960E94DE1291E0811101C090E0F9
:201A6000892F08C040E0BE01C8010E94C41C882311F3EDCFDF91CF911F910F910895FC0197
:201A8000DB0112968D919C911397938382838CE092E09183808314968C9114978483159699
:201AA0008C911597858316964D915D916D917C91199746835783608771871A964D915D9124
:201AC0006D917C911D9742875387648775871E964D915D916D917C91519746875787608BB4
:201AE000718B52968C915297828B53964D915D916D917C915697438B548B658B768B5796B7
:201B00004D915D916D917C915A97478B508F618F728F5B968D919C915C97948F838F08955A
:201B20004F925F926F927F928F929F92AF92BF92CF92DF92EF92FF920F931F93CF93DF93D1
:201B4000CDB7DEB7C754D1090FB6F894DEBF0FBECDBF6C014A013901665D7F4F5E018EE1DF
:201B6000A80EB11CC5010E943F0D1C821B828CE092E09A8389831E828401FE0131967F0181
:201B80005A2C4B2C6FE270E0C8010E9494370097E9F1F80120812F3219F40F5F1F4FF2CF5B
:201BA000801B8D3008F08CE0A82EB12CA501B801CE01CB960E94A637EBE3F0E0EC0FFD1FF3
:201BC000EA0DFB1D1082C7010E94641521E0AE01455C5F4F652D742DC7010E9498168111A5
:201BE00009C0F601138212828CE092E091838083158216C00A0D1B1D852D942D0E946415BD
:201C0000C2015E2C4F2CE92EF82EBCCF08191909F30111830083652D742DC6010E943F0DFE
:201C2000C601C95BDF4F0FB6F894DEBF0FBECDBFDF91CF911F910F91FF90EF90DF90CF9048
:201C4000BF90AF909F908F907F906F905F904F9008959F92AF92BF92CF92DF92EF92FF9288
:201C60000F931F93CF93DF93CDB7DEB7C955D1090FB6F894DEBF0FBECDBF7C016B015A01A0
:201C8000922E9E01285A3F4FCE01CB960E94900D6A960EAD1FAD6A970A0D1B1DF801808195
:201CA00081110AC0BE01655C7F4FCE0101960E943F0D46E052E041C019A218A28CE092E07A
:201CC0009F8F8E8F1BA221968FAD2197811104C0C7010E948F0C37C08250823060F4B60170
:201CE000665D7F4F292DA801CE014E960E949816811110C0EDCF292DA801BE01655C7F4FE6
:201D0000CE014E960E949816882311F3CE01CB960E946415892D867041F049A95AA96BA9E0
:201D20007CA9CE014E960E948114BE01625E7F4FCE0101960E943F0DA801BE016F5F7F4FEF
:201D4000C7010E94560CC701C75ADF4F0FB6F894DEBF0FBECDBFDF91CF911F910F91FF90AA
:201D6000EF90DF90CF90BF90AF909F90089510929C0810929D081092A0081092A20882E037
:201D800090E0A0E0B0E08093A3089093A408A093A508B093A6081092BA081092C4081092F1
:201DA000C3088CE092E09093C2088093C1081092C60808959FB7F8942091140B8091120BC4
:201DC000213019F48DBB9FBF08958FBF08952091140B222399F03FB7F8942091140B213036
:201DE00059F42DB32093120B4DB32091130B209524232DBB3FBF02C03093120B8CBD9DBDF0
:201E000008958EBD00000DB407FEFDCF8EB508958FEF0C94010F61E0FC0184810E94C10A8A
:201E20008091E008882339F01092E0088091140B81110C94DA0E0895CF93DF93EC01809192
:201E4000E008811109C081E08093E0088091E1089091E2080E94E70E60E08C81DF91CF912A
:201E60000C94C10ACF93DF93EC018E81882389F08F8198859C012F5F3F4F38872F838230FA
:201E8000924018F40E94080FF3CFCE010E940B0F1E82DF91CF910895673028F026E1FC019E
:201EA000258380E00895623081F030F4662359F06130B1F480E515C0643059F040F0653072
:201EC00079F482E50EC080E505C081E503C081E508C082E58093E10881E08093E208089581
:201EE00083E58093E1081092E20881E008950F931F93CF93DF93EB010E94BA098B010E944D
:201F0000080F8F3F49F00E94BA09601B710B6C177D07A8F380E001C081E0DF91CF911F91A3
:201F20000F910895CF92DF92FF920F931F93CF93DF9300D000D0CDB7DEB76C01F62E2983E3
:201F40003A834B835C830E94320FC6010E941C0F6CE271E0C6010E94770F8F2D80640E94D0
:201F6000010F08E110E05C814B813A812981DA01C901002E04C0B695A795979587950A9466
:201F8000D2F729833A834B835C830E94010F0850110929813A814B815C81083F8FEF18074C
:201FA00031F7FF2029F0E8E0FE1621F08FEF03C085E901C087E80E94010F10E00E94080F9A
:201FC000F601828787FF04C01F3F11F01F5FF6CF0F900F900F900F90DF91CF911F910F9179
:201FE000FF90DF90CF900895BF92CF92DF92EF92FF920F931F93CF93DF93EC01B62E1B8618
:2020000019861E821D824C830E94BA098B0161E08C810E94880A61E08C810E94C10A0E9443
:20202000D01F82E58093E1081092E2088091E1089091E2080E94E70E2AE0F22E8FEF0E94DC
:20204000010FFA94D9F78091140B81110E94DA0ECE010E941C0F20E030E0A90160E0CE0161
:202060000E94920FF82E8A8781E0F81649F00E94BA09601B710B613D774068F381E04BC0C6
:202080002AEA31E040E050E068E0CE010E94920F82FF02C0FB860DC094E0F92E0E94080F8C
:2020A0008A87FA94D9F78A3A11F082E034C082E08B878B85823031F4C12CD12CE12C80E4E0
:2020C000F82E03C0C12CD12C760120E030E0A90167E3CE010E94920FA701960169E2CE0147
:2020E0000E94920F8A87882349F00E94BA09601B710B613D774048F388E00DC08B858230C5
:2021000031F520E030E0A9016AE3CE010E94920F882381F086E08D83CE010E940B0F80E003
:20212000DF91CF911F910F91FF90EF90DF90CF90BF9008950E94080F807C803C11F483E0DE
:202140008B870E94080F0E94080F0E94080FCE010E940B0F6B2DCE01DF91CF911F910F9130
:20216000FF90EF90DF90CF90BF900C944C0F0F931F93CF93DF93EC010E94BA098B010E9491
:20218000080F8A878F3F49F40E94BA09601B710B6D327140A0F38FE003C08E3F39F08DE038
:2021A0008D83CE010E940B0F80E001C081E0DF91CF911F910F910895CF92DF92EF92FF9261
:2021C0000F931F93CF93DF93EC0169010115110509F462C0C801820F931F8130924008F0AE
:2021E0005DC08E81882371F088819981AA81BB81481759076A077B0729F48F819885C81643
:20220000D90610F5488359836A837B838B85833039F039E0440F551F661F771F3A95D1F7CA
:202220009A01AB0161E1CE010E94920F882319F083E08D8333C0CE010E94B710882371F1A4
:2022400018861F8281E08E838F8198858C159D0540F40E94080F8F819885019698878F837B
:20226000F3CF6701E00EF11ECE14DF0431F00E94080FF60181936F01F7CF8F819885800F9B
:20228000911F98878F832985222319F08115924018F0CE010E94320F81E004C0CE010E94A9
:2022A0000B0F80E0DF91CF911F910F91FF90EF90DF90CF900895EF92FF920F931F9379012B
:2022C00000E012E020E030E00E94DC101F910F91FF90EF900895CF92DF92EF92FF920F930D
:2022E0001F93CF93DF9300D0CDB7DEB78C01862F49835A830E94010F4981C42E5A81D52E38
:20230000E12CF12CF60181916F010E94010FFFEFEF1AFF0AE11482E0F806A1F78FEF0E945B
:20232000010F8FEF0E94010F0E94080FF80182878F71853039F081E18583C8010E940B0FD5
:2023400080E001C081E00F900F90DF91CF911F910F91FF90EF90DF90CF9008950F931F93D0
:20236000CF93DF93EC018901411551056105710511F482E132C08B85833039F089E0440F88
:20238000551F661F771F8A95D1F79A01AB0168E1CE010E94920F882311F084E01EC0A8018E
:2023A0006EEFCE010E946B118823C1F068E572E0CE010E94770F811102C085E10EC020E059
:2023C00030E0A9016DE0CE010E94920F811104C00E94080F882339F084E18D83CE010E941B
:2023E0000B0F80E004C0CE010E940B0F81E0DF91CF911F910F91089580E58093E1081092F3
:20240000E2080895CF93DF93EC019C012A5F3F4F41E050E060E070E08B8D9C8D0E94591B88
:202420008823A1F04F89588D698D7A8D452B462B472B71F44E815F81688579854F8B588F93
:20244000698F7A8F8C8180688C8302C080E001C081E0DF91CF910895CF92DF92EF92FF92E2
:202460001F93CF93DF93EC010E940212811102C080E04BC0EB8DFC8DCE80DF80E884F984DD
:2024800082E0C81AD108E108F108058404C0CC0CDD1CEE1CFF1C0A94D2F746855785608903
:2024A0007189C40ED51EE61EF71E148181E0C81AD108E108F108112361F0C701B601610F3D
:2024C000711D811D911D0E94A319882389F21150F2CFEB8DFC8DC12C82E0D82EE12CF12CFC
:2024E000058404C0CC0CDD1CEE1CFF1C0A94D2F74B895C896D897E894C0D5D1D6E1D7F1D82
:202500004B8B5C8B6D8B7E8B81E0DF91CF911F91FF90EF90DF90CF900895CF93DF93EC01E2
:20252000462F6E857F85888999890E946819882341F08A8920E2829FC00111248451974F16
:2025400002C080E090E0DF91CF910895282FFB018BE030E231938150E9F7A22FB92F20E07E
:2025600037E09D91992319F19E3219F0E8E5F3E008C03A3011F128E03AE0F3CF3196491798
:20258000E1F044914111FACF3217B8F04FED490F4E3598F441E0420FFB01E20FF11D2FE961
:2025A000290F2A3108F490529083242FDACF81E0FB019081903209F480E008950F931F931D
:2025C000CF93DF93EC018B018D81882311F080E040C0FB0187898031B1F482E08D831F8A17
:2025E000188E198E1A8E408D518D60E070E095E0440F551F661F771F9A95D1F74B8B5C8BA0
:202600006D8B7E8B15C0803211F783E08D83FB01428D538D648D758D4F8B588F698F7A8F57
:202620009E012D5E3F4FC8010E944D1A882379F21C8F0B8F81E08C831E821F8218861986C7
:202640001A861B861C861D861E861F86188A198A1A8ADF91CF911F910F9108952F923F9273
:202660004F925F926F927F928F929F92AF92BF92CF92DF92EF92FF920F931F93CF93DF9386
:20268000EC016B015A018D81811103C08FEF9FEFDAC08C8180FFFACF4B895C896D897E8972
:2026A0008A859B85AC85BD852501612C712C8A019B01081B190B2A0B3B0B041515052605E1
:2026C000370518F45A01A81AB90A25011E0126E0220E311C4114510409F47BC04A855B8579
:2026E0006C857D854A0181E09822ED818A019B01F9E03695279517950795FA95D1F78B8DD5
:202700009C8DE23051F4FC01628D738D848D958D600F711F821F931F3EC0FC0174807A94CB
:20272000702281149104C9F4711017C0452B462B472B49F48F89988DA98DBA8D8E839F834B
:20274000A887B9870AC04E815F816885798591010E94C919882309F499CFEB8DFC8D6E8190
:202760007F81888599856250710981099109058404C0660F771F881F991F0A94D2F7068535
:20278000178520893189600F711F821F931F670D711D811D911D20E032E0281939093201D2
:2027A0002415350508F439012C8126FD04C06114F2E07F06A1F50091100110911101209174
:2027C000120130911301601771078207930719F426C0C50138C0760183019401AB01BC0155
:2027E0008091EA089091EB080E94DC10882309F44DCFC60CD71C04C0E81BF90BCE0EDF1E07
:202800008A859B85AC85BD85860D971DA11DB11D8A879B87AC87BD87461857085BCF40E092
:202820000E946819882309F431CFC4018451974FD6019C01260D371DFC01E217F307E1F28F
:2028400041914D93FACFDF91CF911F910F91FF90EF90DF90CF90BF90AF909F908F907F9016
:202860006F905F904F903F902F900895FF920F931F93CF93DF931F92CDB7DEB78C01FC0153
:202880008581823018F480E090E034C0F8014285538564857585A5E07695679557954795E1
:2028A000AA95D1F7F42FFF70FF2E41E050E0BE016F5F7F4FC8010E942E13019719F42981AB
:2028C00030E002C02FEF3FEF2F3F3F4FE1F2F8014285538564857585415E5F4F6F4F7F4FB7
:2028E0004287538764877587F0E2FF9EC00111248451974F0F90DF91CF911F910F91FF90E0
:2029000008954F925F926F927F92AF92BF92CF92DF92EF92FF920F931F93CF93DF93EC01AB
:202920006A017B012D81222309F457C08B899C89AD89BE8984179507A607B70708F44DC048
:202940004EC08A859B85AC85BD85EB8DFC8DE585F0E03996AC01BD01415051096109710983
:202960000E2E04C076956795579547950A94D2F797018601015011092109310904C03695A4
:20298000279517950795EA95D2F70417150726073707B0F58F89988DA98DBA8D8E839F83B7
:2029A000A887B987280139015E0186E0A80EB11C411451046104710461F14E815F8168858B
:2029C000798595018B8D9C8D0E94C91991E0491A5108610871088111EBCF80E01FC02230B2
:2029E000C1F0C114D104E104F10409F0AACF1E821F82188619861A861B861C861D860DC05F
:202A0000892B8A2B8B2B31F2041B150B260B370BC9CFCA86DB86EC86FD8681E0DF91CF9153
:202A20001F910F91FF90EF90DF90CF90BF90AF907F906F905F904F9008950F931F93CF93AD
:202A4000DF93EC018D818823C9F18C8187FF30C061E0CE010E948D128C01009779F18D8134
:202A6000823048F44B895C896D897E89F801448F558F668F778F4F89588D698D7A8DF80154
:202A8000538F428F758B648BE091E308F091E408309759F0B8016A5E7F4FC8014896099527
:202AA000F801808D918D938B828B8C818F778C83DF91CF911F910F910C942D1980E0DF91CF
:202AC000CF911F910F910895CF93DF93EC010E941D15882319F01D8281E001C080E0DF91CF
:202AE000CF9108954F925F926F927F92AF92BF92CF92DF92EF92FF920F931F93CF93DF9357
:202B000000D000D0CDB7DEB75C016A017B01FC0185818130F1F4848181FF1BC0F5018389BD
:202B20009489A589B68984179507A607B70788F0892B8A2B8B2B09F479C0F5014284538409
:202B400064847584B701A601C5010E948114811102C080E06CC0F501838D948DC114D10487
:202B6000E104F10471F44789508D618D728D0E946E1C882371F3F501178A108E118E128ECD
:202B80003AC0F50146815781608571859E012F5F3F4F0E94C9198823E1F249815A816B817D
:202BA0007C81F501838D948DFC012789203129F408EF1FEF20E030E004C008EF1FEF2FEFDA
:202BC0003FE04017510762077307A8F40E946E1C882309F4BECFF5014681578160857185D7
:202BE0000FEF1FEF2FEF3FE0838D948D0E94B81A882309F4AECFF501C38AD48AE58AF68A32
:202C0000848180688483C5010E941D15882309F4A0CFB701A6014C145D046E047F0410F4F6
:202C2000B301A201C5010E94811401C081E00F900F900F900F90DF91CF911F910F91FF90F3
:202C4000EF90DF90CF90BF90AF907F906F905F904F900895FF920F931F93CF93DF93EC017A
:202C6000F42E80E2689FF0011124E451F74F8385817129F0842F827411F080E053C06A8B03
:202C80008091100190911101A0911201B09113018E879F87A88BB98B4489558960E070E059
:202CA000BA0155274427028D138D20E030E0402B512B622B732B4F8B588F698F7A8F838557
:202CC000887151F4048D158D268D378D0B8B1C8B2D8B3E8B81E00CC0803179F69E012D5ED7
:202CE0003F4F8B8D9C8D0E944D1A882331F284E08D838F2D8F708C831E821F821886198672
:202D00001A861B861C861D86F6FE0BC040E050E0BA01CE01DF91CF911F910F91FF900C9445
:202D2000721581E0DF91CF911F910F91FF900895AF92BF92CF92DF92EF92FF920F931F9395
:202D4000CF93DF93CDB7DEB72B970FB6F894DEBF0FBECDBF7C016B01CA01B22EF70125814B
:202D60002111B9C0BE016F5F7F4F0E94A612882309F4B1C0F601838D948DF701948F838F85
:202D8000F60116821782108611861286138614861586A12CF6010285138524853585838926
:202DA0009489A589B689081719072A073B07E8F545E036952795179507954A95D1F70F70E0
:202DC000C6010E943614009709F485C0FC012081222311F0253EB9F4A1100EC0F701028B6F
:202DE0004091100150911101609112017091130146875787608B718BFC018081AA24A39450
:202E00008111C8CF12C04BE050E0BC01CE0101960E948737892B09F0BDCF8B2D8073803342
:202E200009F459C04B2D602F52C08B2D8271823109F051C0AA2041F061E0C7010E948D12B6
:202E40008C01009779F447C0F6018581823009F442C0C6010E942C128823E9F1F701128A6C
:202E60000CEE18E080E2F80111928A95E9F78BE0FE013196D80101900D928A95E1F7E091C1
:202E8000E308F091E408309739F0B801625F7F4FC8014096099509C081E298E2F801918BAA
:202EA000808B80E098E097878687F80180899189938B828B918F808F86859785978B868B34
:202EC0000E942D19882339F04B2DF7016289C7010E942A1601C080E02B960FB6F894DEBF61
:202EE0000FBECDBFDF91CF911F910F91FF90EF90DF90CF90BF90AF9008952F923F924F92DF
:202F00005F926F927F928F929F92AF92BF92CF92DF92EF92FF920F931F93CF93DF9300D0EE
:202F200000D01F92CDB7DEB78C017B013A01DC0115968C9115978130C9F414968C9181FFAD
:202F400015C082FF1BC0F801438954896589768982859385A485B58584179507A607B7078D
:202F600069F0C8010E948114811108C081E090E0F8019383828380E090E046C1630180C03E
:202F8000D8015B968D919C915C97FC01F481F150B501A40129E076956795579547952A9584
:202FA000D1F7F423FD8321E09222FF2309F474C080E092E08819990956018C159D0508F4FF
:202FC0005C01D8015B96ED91FC915C9716962D903D904D905C901997B2E02B1A31084108C4
:202FE0005108058404C0220C331C441C551C0A94D2F786859785A089B189280E391E4A1EF7
:203000005B1EED812E0E311C411C511CA114F2E0BF0609F088C08091100190911101A09163
:203020001201B091130182159305A405B50559F48FEF9FEFDC018093100190931101A093D4
:203040001201B09313019701B201A1018091EA089091EB080E94AE11882309F487CF9EEF16
:20306000F91ACA18DB08F80182859385A485B5858A0D9B1DA11DB11D82879387A487B58798
:20308000D8011A968D909D90AD90BC901D97C114D10409F075CF8AC08114910409F088CF75
:2030A00016964D915D916D917C911997411551056105710559F457968D919D910D90BC91E5
:2030C000A02D0097A105B10541F521C09E012F5F3F4F0E94C919882309F44ECF89819A81F0
:2030E000AB81BC81F801238D348DF9012789203129F448EF5FEF60E070E004C048EF5FEF87
:203100006FEF7FE084179507A607B70730F0C8010E94021281114CCF29CFF80186839783F0
:20312000A087B18745CF8114910429F5D8011A964D915D916D917C911D9753968D919D918B
:203140000D90BC91A02D481759076A077B0798F00E942D19882309F409CF20921001309291
:20316000110140921201509213018091E90881608093E90808C041E0C201B1010E946819FA
:20318000882309F4F3CEC4018451974FD7019C012A0D3B1DFC01E217F30719F04D91419397
:2031A000FACFE81BF90BEE0EFF1E5BCF53968D919D910D90BC91A02DF80124818815990537
:2031C000AA05BB0538F4838A948AA58AB68A206824830CC08091E3089091E408892B31F0E1
:2031E0006114710419F02068F8012483D80114968C9183FD02C0C30107C0C8010E941D15AA
:20320000882309F4B3CEF7CF0F900F900F900F900F90DF91CF911F910F91FF90EF90DF9007
:20322000CF90BF90AF909F908F907F906F905F904F903F902F900895CF93DF931F92CDB743
:20324000DEB7698341E050E0BE016F5F7F4F0E947D170F90DF91CF9108958091E908882352
:2032600099F1409110015091110160911201709113012CEE38E08091EA089091EB080E94EB
:20328000AE11882319F14091E5085091E6086091E7087091E808411551056105710591F053
:2032A0002CEE38E08091EA089091EB080E94AE11882361F01092E5081092E6081092E708B8
:2032C0001092E8081092E90881E0089580E00895CF92DF92EF92FF92CF936B017C01C42FAC
:2032E0008091100190911101A0911201B09113018C159D05AE05BF05D1F00E942D198111EB
:2033000002C080E01AC02CEE38E0B701A6018091EA089091EB080E945B11882391F3C0927A
:203320001001D0921101E0921201F09213018091E9088C2B8093E90881E0CF91FF90EF9061
:20334000DF90CF900895CF92DF92EF92FF926B017C010E942D198823B1F0ECEEF8E01192AC
:203360008AE0EC3EF807D9F7C0921001D0921101E0921201F09213018091E9088160809302
:20338000E90881E001C080E0FF90EF90DF90CF9008958F929F92AF92BF92CF92DF92EF920A
:2033A000FF920F931F93CF93DF938C016A017B01E901FC0181859285A385B4850196A11D26
:2033C000B11D84179507A607B70710F480E058C0F80143895489658976898789803129F494
:2033E000BB27AF2D9E2D8D2D09C0D701C60127E0B695A795979587952A95D1F74C015D011A
:20340000840E951EA61EB71EC501B4018090100190901101A0901201B0901301681579056E
:203420008A059B0589F4F8018789803199F4DD24EE24FF24F601EE0FFF1FE451F74F8081D5
:203440009181A0E0B0E017C040E00E9468198111EACFBCCFE894C7F8DD24EE24FF24F601F2
:20346000EE0FFF1FEE0FFF1FE451F74F80819181A281B381BF7088839983AA83BB8381E00F
:20348000DF91CF911F910F91FF90EF90DF90CF90BF90AF909F908F9008954F925F926F92E4
:2034A0007F92AF92BF92CF92DF92EF92FF920F931F93CF93DF9300D000D0CDB7DEB78C0117
:2034C00049835A836B837C835901C12CD12C7601412C42E0542E612C712C49815A816B81CF
:2034E0007C819E012F5F3F4FC8010E94C919882359F1D301C201F801058404C0880F991FA6
:20350000AA1FBB1F0A94D2F7C80ED91EEA1EFB1E49815A816B817C818789803129F488EFD0
:203520009FEFA0E0B0E004C088EF9FEFAFEFBFE0481759076A077B0780F2F501C082D18238
:20354000E282F38281E001C080E00F900F900F900F90DF91CF911F910F91FF90EF90DF90F7
:20356000CF90BF90AF907F906F905F904F9008954F925F926F927F928F929F92AF92BF921D
:20358000CF92DF92EF92FF920F931F93CF93DF93EC016A017B0128013901423051056105BA
:2035A000710508F474C049855A856B857C854F5F5F4F6F4F7F4F4C155D056E057F0508F429
:2035C00066C08B889C88AD88BE888F89803129F477276F2D5E2D4D2D09C0B701A601E7E0FF
:2035E0007695679557954795EA95D1F7840E951EA61EB71E409110015091110160911201FE
:203600007091130184169506A606B70671F48F89803199F4DD24EE24FF24F601EE0FFF1FF4
:20362000E451F74F5182408218C040E0C501B4010E9468198111EBCF2AC0E894C7F8DD2472
:20364000EE24FF24F601EE0FFF1FEE0FFF1FE451F74F40825182628273828091E90881603C
:203660008093E9088A89823080F08D819E81AF81B885880D991DAA1DBB1D8093E50890936A
:20368000E608A093E708B093E80881E001C080E0DF91CF911F910F91FF90EF90DF90CF9069
:2036A000BF90AF909F908F907F906F905F904F9008952F923F924F925F926F927F929F920E
:2036C000AF92BF92CF92DF92EF92FF920F931F93CF93DF93CDB7DEB760970FB6F894DEBF4E
:2036E0000FBECDBF5C014D875E876F87788B1901D9014D905D906D907C904114510461048C
:20370000710431F0BFEF4B1A5B0A6B0A7B0A10C0FC014080518062807380992493940D85F8
:203720001E852F853889013011052105310509F0912CD50119962D913D914D915C911C9789
:203740002F5F3F4F4F4F5F4F29873A874B875C87730162011D821E821F821886F50181858A
:203760009285A385B4850D811E812F813885081719072A073B0708F056C029853A854B853A
:203780005C852C153D054E055F0550F4A2E0CA2ED12CE12CF12CB2E04B2E512C612C712C77
:2037A0009E012F5F3F4FB701A601C5010E94C9198823C9F149815A816B817C81D701C60113
:2037C0000196A11DB11D452B462B472B19F02C013D010FC0AC01BD0144195509660977091B
:2037E0000D851E852F853889401751076207730779F02D813E814F8158852F5F3F4F4F4F50
:203800005F4F2D833E834F8358876C017D01A6CF0FEF1FEF2FEF3FE0B701A601C5010E9468
:20382000B81A811118C080E041C0D701C6010197A109B1098D839E83AF83B887970186018F
:20384000AC01BD01C5010E94B81A882361F3CD80DE80EF80F8844C145D046E047F0428F35D
:20386000D1014D915D916D917C91411551056105710599F4F1014082518262827382992071
:20388000A1F0FFEF4F1A5F0A6F0A7F0AD5014D925D926D927C92139708C093018201C501D5
:2038A0000E94B81A8111E6CFBECF81E060960FB6F894DEBF0FBECDBFDF91CF911F910F9102
:2038C000FF90EF90DF90CF90BF90AF909F907F906F905F904F903F902F900895AF92BF92B6
:2038E000CF92DF92EF92FF920F931F93CF93DF9300D000D0CDB7DEB75C016A017B0182E05D
:2039000090E0A0E0B0E0F50180839183A283B3839E012F5F3F4FB701A601C5010E94C9195B
:20392000882311F100E010E09801B701A601C5010E94B81A8823C1F0C980DA80EB80FC80F2
:20394000F5018789803129F488EF9FEFA0E0B0E004C088EF9FEFAFEFBFE0C816D906EA06CB
:20396000FB06B0F281E001C080E00F900F900F900F90DF91CF911F910F91FF90EF90DF9009
:20398000CF90BF90AF9008958F929F92AF92BF92CF92DF92EF92FF920F931F93CF93DF93AD
:2039A000EC01142F7093EB086093EA08442341F1453010F080E0EFC040E060E070E0CB0163
:2039C0000E9468198823B1F320E1129FF0011124E656F54F80818F7769F784859585A68568
:2039E000B78584369105A105B10520F3C084D184E284F384C114D104E104F10421F4DACF14
:203A0000C12CD12C760140E0C701B6010E946819882381F28091F7089091F80881159240CC
:203A200049F63091FC08332329F28091FA089091FB08892B09F4BECF2091F908222309F4A8
:203A4000B9CF3A8B2C831D8630E041E050E06D85062FCA01062E02C0880F991F0A94E2F7B8
:203A60002817390731F081E0860F8D87683078F3A1CF20910209309103092115310519F02B
:203A800040E050E008C0209110093091110940911209509113092D833E834F83588780914D
:203AA000FA089091FB0846015701880E991EA11CB11C8B8A9C8AAD8ABE8AE091FD08F091B9
:203AC000FE08F98FE88FA091FC08B0E00E947D38680D791D8A1D9B1D6A8F7B8F8C8F9D8F11
:203AE00015E0EE0FFF1F1A95E1F7E150FE4FEF2FFF27E695DC01CB018E0F9F1FA11DB11D62
:203B00008E879F87A88BB98B8090FF08909000098114910419F0A12CB12C08C080900C09E9
:203B200090900D09A0900E09B0900F09A7019601281B390B4A0B5B0BDA01C901880D991D3F
:203B4000AA1DBB1D04C0B695A795979587950A95D2F789879A87AB87BC87853F3FE09307A8
:203B6000A105B10510F48CE014C0853F9F4FA105B10510F480E10DC08091180990911909F0
:203B8000A0911A09B0911B098A8F9B8FAC8FBD8F80E28F8B81E0DF91CF911F910F91FF9016
:203BA000EF90DF90CF90BF90AF909F908F9008951F920F920FB60F9211240BB60F922F932E
:203BC0003F934F935F936F937F938F939F93AF93BF93EF93FF938091ED0A87FF05C010923A
:203BE0008500109284001AC02091ED0A332727FD30958091EC0A90E0281739077CF48091DE
:203C0000ED0A992787FD9095FC01EE0FFF1FE80FF91FE251F54F808186FD15C08091ED0A45
:203C20008F5F8093ED0A2091ED0A332727FD30958091EC0A90E028173907BCF48091ED0AF3
:203C40008C305CF112C08091ED0A992787FD9095FC01EE0FFF1FE80FF91FE251F54F808179
:203C600060E08F730E94C10AD9CF8091840090918500049680349C4918F480E49CE905C0C5
:203C80008091840090918500049690938900809388008FEF8093ED0A38C020918400309192
:203CA00085008091ED0A992787FD9095FC01EE0FFF1FE80FF91FE251F54F81819281820FCA
:203CC000931F90938900809388008091ED0A992787FD9095FC01EE0FFF1FE80FF91FE25120
:203CE000F54F808186FF11C08091ED0A992787FD9095FC01EE0FFF1FE80FF91FE251F54F1A
:203D0000808161E08F730E94C10AFF91EF91BF91AF919F918F917F916F915F914F913F9152
:203D20002F910F900BBE0F900FBE0F901F9018952091EC0A2C30A0F431E0320F3093EC0A52
:203D4000FC012083822F90E0FC01EE0FFF1FE80FF91FE251F54F88EB9BE092838183089560
:203D60002FEFFC0120830895DF92EF92FF920F931F93CF93DF93EC01D62E7A01890188813E
:203D80008C3008F066C061E08D2D0E94880A8881A82FB0E0FD01EE0FFF1FEA0FFB1FE2514B
:203DA000F54F2D2D2F739081907C922B908360E272E06E197F0977FF02C06D5F7F4F759557
:203DC000679575956795698340E659E0401B510B57FF02C04D5F5F4F5595479555954795E1
:203DE0004A836CE00E9416389CE0899FB001112420E030E0A901460F571FFA01EE0FFF1F95
:203E0000E40FF51FE251F54F908196FD16C02F5F3F4F2C30310571F781110FC01092800011
:203E200082E0809381001092850010928400B19A80916F00826080936F00888190E0FC019A
:203E4000EE0FFF1FE80FF91FE251F54F8081806480838881DF91CF911F910F91FF90EF90A2
:203E6000DF90089520E639E040E252E00C94B41EFC0180818C3070F5918128E830E0291BBC
:203E8000310997FD3395220F331F220F331F621773077CF0928128E532E0291B310997FDE3
:203EA0003395220F331F220F331F621773070CF49B0122503109220F331F4FB7F89490E074
:203EC000FC01EE0FFF1FE80FF91FE251F54F328321834FBF08954F925F926F927F92AF921B
:203EE000BF92CF92DF92EF92FF920F931F93CF93DF93EC01603282E078070CF040C077FD95
:203F000006C0653B71052CF064EB70E002C060E070E0898128E830E0281B310987FD3395C5
:203F2000220F331F220F331F5901CC24B7FCC094DC2C882777FD8095982F2A8148E552E019
:203F4000421B510927FD5395440F551F440F551F2A01662457FC6094762C7F926F925F926F
:203F60004F9214EBE12EF12C00E010E020E030E0A9010E94DB350F900F900F900F90CE01AE
:203F8000DF91CF911F910F91FF90EF90DF90CF90BF90AF907F906F905F904F900C94381FC4
:203FA000CF93CFB7F8948091150B811127C0E8E2F3E08491E8E0F3E09491E82FF0E0EE0F8D
:203FC000FF1FE25BFC4FA591B4918C91892321F461E084E00E94C10A61E084E00E94880AF7
:203FE0008CB580618CBD8CB580648CBD61E087E00E94880A61E085E00E94880A8091150B01
:204000008F5F8093150BCFBFCF9108952F923F924F925F926F927F928F929F92AF92BF929A
:20402000CF92DF92EF92FF920F931F93CF93DF9300D000D0CDB7DEB74C017C836B836A0116
:204040005901C8018701AC014C195D0957FF03C051954195510995016B817C81261B370B0C
:2040600037FF03C031952195310922242394312C2417350714F0212C312C2114310459F05F
:204080003A2D2B2D5C01832F922F3B812C81DC82CB82C32ED22EAB81BC81AA16BB065CF452
:2040A0003C2D2D2D6C01832F922F3B812C81BC82AB82A32EB22E2501EB81FC814E1A5F0AF8
:2040C0003C016C187D0877FE03C0719461947108720157FE03C0FFEFEF1AFF0AF594E79460
:2040E000C816D9062CF421E030E03A83298324C06FEF7FEF7A8369831FC0D401ED91FC9111
:204100000480F581E02D980121143104D9F04B815C81B601C4010995E618F708F7FE06C051
:20412000E981FA81CE0EDF1EE40CF51C2B813C812F5F3F4F3C832B836B817C81A616B7066C
:20414000E4F604C0A6016B817C81E4CF0F900F900F900F90DF91CF911F910F91FF90EF90D4
:20416000DF90CF90BF90AF909F908F907F906F905F904F903F902F9008956F927F928F925B
:204180009F92AF92BF92CF92DF92EF92FF920F931F93CF93DF93EC015B016A013901480119
:2041A000E881F9810284F385E02D87010995E881F981A601480D591D415051090284F385AD
:2041C000E02D9301B501CE010995E881F9810084F185E02D9401A601B501CE010995E88169
:2041E000F981B501660D771D615071090084F185E02D9401A601CE010995DF91CF911F912D
:204200000F91FF90EF90DF90CF90BF90AF909F908F907F906F900895EF92FF920F931F9335
:20422000DC01ED91FC91240F351F215031090680F781E02D780189019B0109951F910F91CC
:20424000FF90EF900895EF92FF920F931F93DC01ED91FC91260F371F215031090680F78131
:20426000E02D78018A0109951F910F91FF90EF9008956F927F928F929F92AF92BF92CF923D
:20428000DF92EF92FF920F931F93CF93DF935C014A0169013801EB01C60ED71ECC15DD05B0
:2042A00074F4D501ED91FC910084F185E02D87019301A401BE01C50109952196EFCFDF91E5
:2042C000CF911F910F91FF90EF90DF90CF90BF90AF909F908F907F906F900895EF92FF92B9
:2042E0000F931F93DC01ED91FC9111971A960D911C911B9718962D913C9119970684F7853E
:20430000E02D7B0140E050E060E070E009951F910F91FF90EF9008950895CF92EF92FF928B
:204320000F931F93CF93DF93EC01262F6A3049F42C898E859F8538E0239F800D911D112406
:2043400036C06D30C1F1E881F981EA88FB88088919894E855F856C857D850488F589E02D4C
:20436000CC8809952C89422F50E08C859D8536E0239F800D911D11249D878C872E89222347
:20438000D1F06AEF64039001659F300D112468857985260F371F281739076CF473E0440F9A
:2043A000551F7A95E1F78E859F85840F951F9F878E871D861C8681E090E0DF91CF911F9153
:2043C0000F91FF90EF90CF900895CF92EF92FF920F931F93CF93DF93EC01262F6A3049F47F
:2043E0002C898E859F8538E0239F800D911D112436C06D30C1F1E881F981EA88FB880889D9
:2044000019894E855F856C857D850488F589E02DCC8809952C89422F50E08C859D8537E0A7
:20442000239F800D911D11249D878C872E892223D1F069EF64039001659F300D11246885A3
:204440007985260F371F281739076CF4E3E0440F551FEA95E1F78E859F85840F951F9F876F
:204460008E871D861C8681E090E0DF91CF911F910F91FF90EF90CF9008952F923F924F9274
:204480005F926F927F928F929F92AF92BF92CF92DF92EF92FF920F931F93CF93DF93CDB7A5
:2044A000DEB72C970FB6F894DEBF0FBECDBF9C878B873A011F830E83F986E886CA86DC01A0
:2044C00018968D919C911997681779070CF08BC01A968D919C911B97481759070CF083C042
:2044E000AC2CB12CC501F3E0880F991FFA95E1F7AB01480F591F141615060CF074C0860D35
:20450000971D181619060CF06EC04B01B8E02B9F20011124461A570A6B011D82F201E8596C
:20452000FC4F2F01F201E80DF91D24912C837A82698213011B823C8130FF13C0AB85BC85D6
:20454000ED91FC91BA85B13031F40480F581E02D2E813F8119C00684F785E02DEE80FF80BC
:204560001FC0E885F9852E813F81E217F307F9F0AB85BC85ED91FC91BA85B13061F40480B1
:20458000F581E02D2885398549815A81B4018B859C8509950CC00684F785E02DE884F9843C
:2045A00085019501A101B6018B859C850995EC81E695EC83FB81FF5FFB8329813A812F5F15
:2045C0003F4F3A8329832A0C3B1CF83009F0B3CF3D813F5F3D838FEF881A980ACA0CDB1C09
:2045E000383009F09FCF2C960FB6F894DEBF0FBECDBFDF91CF911F910F91FF90EF90DF9046
:20460000CF90BF90AF909F908F907F906F905F904F903F902F900895FC011382128284E1CD
:2046200092E09183808375836483578346837187608753874287158A1586148617861686E0
:2046400021E0248B8FEF9FEF938B828B918B808B268B0895FC0175876487578746870895D2
:20466000611101C061E0FC01648B0895FC01738B628B718B608B0895E091190BF0911A0B96
:204680009F012F5F3F4F30931A0B2093190B808308951F93CF93DF93C62FD72F182F160F12
:2046A0001C1721F089910E943C23FACFDF91CF911F910895CF93DF93EC0186E191E0EAE64C
:2046C000F2E0DF019C011D9221503040E1F780912B0B833019F460E47BE002C06CE272E01B
:2046E00043E450E084E490E00E94B12B6CE272E08AE692E00E94D62F81E0809394028093C7
:20470000950286E0809396024091270B5091280B6091290B70912A0B409398025093990294
:2047200060939A0270939B0280912B0B833031F460E57BE080EA92E00E94CB2F64E57BE06F
:2047400080EB92E00E94D62F80E893E090931A0B8093190B64E171E086E00E944923809160
:204760002B0B811102C081E001C083E00E943C238DE30E943C2387E00E943C2381E00E944D
:204780003C2364E57BE086E00E9449238CE00E943C238AE00E943C236AE171E08AE00E9422
:2047A00049232097A9F082E30E943C2384E00E943C23BE0184E00E94492386E30E943C23D7
:2047C00084E00E943C2360E47BE084E00E944923C091180BC11102C0D3E001C0D4E087E3C9
:2047E0000E943C238D2F0E943C2381E00E943C2383E00E943C2386E00E943C23CC2319F0D6
:204800008C2F0E943C238FEF0E943C238091190B90911A0B84599240DF91CF910C94102C87
:204820000F931F93A62F8634910580F120918D02233461F5009198021091990220919A02ED
:2048400030919B024091270B5091280B6091290B70912A0B0417150726073707B9F4E4E86D
:20486000F3E086599D4F9F012E5F3F4F41815081553319F452815A1739F0F901E40FF11D4F
:20488000E817F90780F302C081E001C080E01F910F910895DF92EF92FF920F931F93CF933C
:2048A000DF9300D000D0CDB7DEB78C0180912B0B823009F497C030F48823D1F1813009F4B4
:2048C00052C031C1833021F0843009F48BC02BC180911B0B90911C0BA0911D0BB0911E0BE6
:2048E0008F3F9F4FAF4FBF4F09F41DC10E94BA0900911F0B1091200B2091210B3091220B5E
:20490000601B710B820B930B00911B0B10911C0B20911D0B30911E0B601771078207930721
:2049200008F401C180E59BE00E945A2384E0EFC00E94BA096093270B7093280B8093290BA0
:2049400090932A0B1092500B1092510B1092520B1092530B80E090E00E945A2381E00E9413
:204960008A2881E0D4C062E0C8010E941024882311F164EA72E0CE0101960E94CB2FE4E894
:20498000F3E006591D4FBF016E5F7F4F81819081963329F480E49BE00E94CB2F06C0FB01E8
:2049A000E80FF11DE017F10770F3CE0101960E945A2382E0ACC00E94BA090091230B109188
:2049C000240B2091250B3091260B601B710B820B930B613177428105910508F4A4C010924A
:2049E0002B0BA1C065E0C8010E941024882319F381E00E949B2864EA72E080E59BE00E949D
:204A0000CB2FE4E8F3E0C80186599D4F7C0180818F010E5F1F4FD1808630B1F048F48130EB
:204A200079F0833009F044C0B80184E49BE00FC08A3381F08F3F09F44AC08333C9F50AC0B1
:204A4000B8018CE49BE003C0B8018CE39BE00E94CB2F3BC0F80184E040E050E0BA0191912B
:204A60002227342F452F562F290F311D411D511D815019F0BA01A901F2CF20931B0B3093A3
:204A80001C0B40931D0B50931E0B2F3F9FEF390749075907D1F0A8EEB3E00E947D386093C8
:204AA0001B0B70931C0B80931D0B90931E0B0DC0E091160BF091170B309739F09091180BE9
:204AC000891303C04D2DB801099580E001C081E0F801ED0DF11D811104C0EE15FF0508F4CA
:204AE00096CF0E94BA0960931F0B7093200B8093210B9093220B8091440B882321F084E48E
:204B00009BE00E942E2C83E080932B0B0CC080932B0B0E94BA096093230B7093240B809392
:204B2000250B9093260B0F900F900F900F90DF91CF911F910F91FF90EF90DF900895CF93D9
:204B4000DF9321E02093370B009781F040E250E0662331F0BC018AE191E00E94A63721C0F0
:204B6000BC018AE191E00E9478371BC02091590B822F90E034E0959587953A95E1F78A307F
:204B800014F430E301C037E3830F80932201822F8F708A3014F490E301C097E3890F80938C
:204BA000230110922B0B0E94BA09EB0180912B0B833069F40E943A2C1092350B1092340B86
:204BC00081E090912B0B933091F080E010C00E94BA096C1B7D0B60367A4E60F70E94BF27F8
:204BE000882321F30E9420280E944A24DFCFDF91CF9108958EBD0DB407FEFDCF089561E026
:204C000080912F0B0E94C10A78940895F89460E080912F0B0C94C10A1F93CF93DF9300D05B
:204C2000CDB7DEB7182F4A8369830E9406266981862F8F71812B0E94FA254A81842F0E9461
:204C4000FA250F900F90DF91CF911F910C94FF251F93CF93DF93182F1076C12FD0E020910F
:204C6000300B30E0C217D307A1F043E06FE180EA0E940C261093300BAE0185E0559547953C
:204C80008A95E1F76FE180E8DF91CF911F910C940C26DF91CF911F9108951F93CF93DF9370
:204CA0001F92CDB7DEB7182F69830E9428264981612F80E40F90DF91CF911F910C940C2658
:204CC0001F93CF93DF931F92CDB7DEB7182F79830E944D267981672F81E0810F0F90DF919C
:204CE000CF911F910C944D260F931F93CF93DF93EC018B010E940626209731F4DF91CF9176
:204D00001F910F910C94FF258AE70E94FA25F80181918EBDC00FD11FEC17FD0731F08191FE
:204D20000DB407FEFDCF8EBDF7CF0DB407FEFDCFE5CF0F931F93CF93DF93EC018B010E9447
:204D400006262097B9F08AE30E94FA251EBCF801CE01019739F00DB407FEFDCF2EB51EBCE7
:204D60002193F7CF2197C00FD11F0DB407FEFDCF8EB58883DF91CF911F910F910C94FF257E
:204D80001F93CF93DF931F92CDB7DEB7182F0E940626812F8F710E94FA2580E00E94FA251C
:204DA00017FF03C080E00E94FA258EB589830E94FF2589810F90DF91CF911F910895CF93BC
:204DC000C82F0E9428268C2FCF910C94C02661E084E00E94880A61E084E00E94C10A61E01F
:204DE00085E00E94880A61E087E00E94880A60E086E00E94880A61E085E00E94C10A60E011
:204E000085E00E94C10A60E087E00E94C10A80E58CBD8DB581608DBD08950F931F93CF933E
:204E2000DF931F92CDB7DEB78B019093330B8093320B0CB406FC04C049830E94E72649812E
:204E400040932F0B61E0842F0E94880A0E94FF254FEF60E08FEF0E940C2662E070E080E095
:204E600090E00E94E9098DE10E94C0268823D9F360E070E088E00E94602660E070E08CE0A5
:204E80000E9460266FEF7BE08AE00E94602660E07CE084E00E9460266FEF71E186E00E94BF
:204EA000602661EB88E30E944D266FE370E388E20E94602669EF77EF80E30E9460266DE0D3
:204EC00080EC0E944D2660E081EC0E944D2642E362EC80E80E940C2662E17CE086EC0E942D
:204EE000602662E184EC0E944D266CED75E08AEC0E946026F801608184EE0E944D26F801BE
:204F0000618185EE0E944D26F801628182EE0E944D26F801638183EE0E944D26F801648185
:204F200080EE0E944D26F801658181EE0E944D2660E184ED0E944D2660E071E086ED0E941E
:204F400060268AEE0E94DF2680FDFBCF8FE10E94282640EC6BE180E80E940C2644E06FE1DD
:204F600080E80E940C2682E70E94DF26863008F08F5F0F90DF91CF911F910F91089561E1AB
:204F800084ED0E944D2661E082ED0E944D268AEE0E94DF2680FDFBCF60E082ED0E944D269C
:204FA00089ED0E94DF2682FB882780F90895CF93DF93EC0140E86FE180E80E940C2640E8F5
:204FC0006FE180EA0E940C264AE06CE180EA0E940C2660E07CE082E00E946026BE01745FD6
:204FE00086E00E94602640E060E08AE70E940C266AE672E0CE010E94742648E06FE180E8F1
:205000000E940C26C0E0D0E08CE10E94DF268A7029F42196C83E83E0D807B1F78CE10E948B
:20502000DF2681FD03C0C83ED34038F048E06FE180EADF91CF910C940C26DF91CF910895F8
:205040000F931F93CF93DF9300D000D000D0CDB7DEB780912E0B882389F060912C0B709108
:205060002D0B6115710519F46FEF7BE002C0615071098CE00E94602610922E0B89E30E94DC
:20508000DF268823C9F160912C0B70912D0B80E00E946026BE016F5F7F4F86E090E00E94EA
:2050A000992689819A8190932D0B80932C0B8B819C810091320B1091330B2D8127FF0DC0F0
:2050C0000497015011098017910708F48C016AE672E0C8010E94992602C000E010E0F801BB
:2050E000E659FD4F108281E080932E0B40E46EE180E80E940C2602C000E010E0C801269620
:205100000FB6F894DEBF0FBECDBFDF91CF911F910F910895CF93C82F88E30E94DF26682F89
:20512000616088E30E944D26C11103C081E08093310BCF910895811102C01092310B8091A9
:20514000310B811108C088E30E94DF26682F6E7F88E30C944D260895CF93DF93EC01FB014B
:205160008A30910548F06AE070E00E942238CB01BF010E94AC28FC01CE016AE070E00E9407
:205180002238805D80831182CF010196DF91CF910895E82FF0E093E0F595E7959A95E1F707
:2051A000E65AF44F877041E050E060E070E004C0440F551F661F771F8A95D2F78081842B56
:2051C00080830895CF93C8E3C15021F08C2F0E94C928FACFCF910895AF92BF92CF92DF9288
:2051E000EF92FF920F931F93CF93DF93CDB7DEB70D851E85EF84F8885E0121E1A20EB11C56
:20520000C7010196F7014491442309F4D9C0443279F0D8011696ED91FC9117979F012F5F1A
:205220003F4F17963C932E93169740837C01E8CFB2E0EB0EF11CFC018491863409F473C06B
:2052400064F48434C9F0853409F09DC0F50180819181F2E0AF0EB11C7EC0D80116964D9170
:205260005C9117978C3409F446C0833509F450C0883409F088C00DC06501B2E0CB0ED11C83
:20528000F80166817781D5018D919C910E94AC2888C095012E5F3F4FF5016081862F99275A
:2052A00087FD9095E4E095958795EA95E1F78F70962F9F709A300CF0995F70E3D72ED90E14
:2052C0008A300CF0895FBA016F5F7F4FD80117967C936E931697805DFA0180831696ED9191
:2052E000FC911797CF01019617969C938E931697D082590185CF6501F4E0CF0ED11CD50188
:205300006D917D918D919C912AE00E94B53749C06501B2E0CB0ED11CF50160817181CA0143
:205320000E949F373EC0F5010190F081E02D22E0A20EB11C2491AF014F5F5F4F222309F470
:205340005FCFF801A681B781CD010196978386832C93FA01EFCF6C01BFEFCB1ADB0A0E9440
:20536000EE37882309F44CCFD8011696ED91FC9117979F012F5F3F4F17963C932E93169761
:205380008083C601E8CFD8011696ED91FC9117979F012F5F3F4F17963C932E9316978083A5
:2053A0002FCFD8011696ED91FC91179701900020E9F731971796FC93EE931697560120CFA8
:2053C000DF91CF911F910F91FF90EF90DF90CF90BF90AF9008950F931F93CF93DF9300D0AE
:2053E0001F92CDB7DEB78C011092370B88E34B8369837A830E94E22869817A8184E59BE0DB
:205400000E94D62F4B8164E57BE0C8010F900F900F90DF91CF911F910F910C940D270F9339
:205420001F93CF93DF9370E066597D4F213021F48A01075F1F4F05C0223031F48A0102502D
:20544000110920E030E003C000E010E09801DB01FA01E230F10578F0CC91D0E0DC2FCC27A4
:2054600011969C911197C92B0C0F1D1F211D311D12963297EECFDA01AE7FA60FB71F40FFD9
:205480000CC04C9150E060E070E0762F652F542F4427040F151F261F371FA90166277727C5
:2054A000411551056105710519F022273327F1CF00951095E82FF0E0E659FD4F1083018335
:2054C000DF91CF911F910F910895109282021092830280E480937E0210927F028093800213
:2054E00020E044E150E06EE088E10C940F2A20918E0230918C0230938E0220938C022091F2
:205500008F0230918D0230938F0220938D02E4E9F2E0A8E9B2E02291820F911D2E918C9382
:20552000662311F0208301C01082892F992722E0E039F20781F710929C0210929D0280E501
:20554000809398020895CF93DF93EC01889690937A0280937B020E94652A10929C021092E0
:205560009D02AE01445E5F4F22E06AE182E30E940F2ACE01C696DF91CF910C94D727BC01AA
:205580008AE692E00E94D62F64E57BE080E792E00C94D62F80E792E00E94BF2A64E872E05E
:2055A00088E892E00E94CB2F60E57BE084E892E00E94CB2F0C94652A262F20612093990200
:2055C000643021F0009711F481E090E061E00E94772A10927A0288E280937B020E94CA2A87
:2055E00084E080939A0210929B0222E04CE150E06AE182E30E940F2A86E390E00C94D727F8
:20560000CF93DF9300D0CDB7DEB769837A830E94BF2A69817A8188E892E00E94CB2F60E5B1
:205620007BE084E892E00F900F90DF91CF910C94CB2F1F93CF93DF93EC018CE292E00E9494
:20564000BF2A88E08093760216E01093770248E050E061E77BE088E792E00E946F37EAE866
:20566000F2E0DF011D921A95E9F764E57BE080E892E00E94D62FBE0180E992E00E94CB2FDF
:2056800060E57BE086E892E00E94CB2F8AE290E0DF91CF911F910C94D727CF93DF93EB0134
:2056A00044E050E0BC0186E892E00E948737892B39F460E872E0CE010E94D62F81E001C086
:2056C00080E0DF91CF910895CF93DF932091500B2223A9F0FC012081222389F0E0E5FBE043
:2056E000EC01ACE4BBE0219189919D918227892331F48BE0E435F807B1F781E001C080E071
:20570000DF91CF91089580917A0290E0982F882720917B02822B44972091980230E064E054
:20572000359527956A95E1F7220F331F220F331F821B930B97FF02C080E090E00895CF93A4
:20574000DF93EC0160E08091610B9091620B0E94DC2A89E180939902CE01DF91CF910C94A0
:20576000A32ACF92DF92EF92FF920F931F93CF93DF93F82EE92EEB01D42EC52ECB010E94C4
:20578000642BBE01882319F08EE69BE002C084E69BE00E94002B2881207F203E91F00881F4
:2057A00019812A813B810F3F1F4F2F4F3F4F49F044E050E0BE0188E49BE00E948737892BD9
:2057C00031F46CE272E08AE692E00E94D62F88E0809376021092770249E050E068E67BE06B
:2057E00088E792E00E946F3710927A0281E180938102C0928E02D0928F02E0928C02F09213
:205800008D02109290021092920210929302DF91CF911F910F91FF90EF90DF90CF900895BF
:20582000CF93DF93EC014C9690937A0280937B020E94652ACE01089690939002809391029D
:20584000AE01405F5F4F21E06AE188E20E940F2ACE018A96DF91CF910C94D7271092350B7C
:205860001092340B21E02093630BBC0184E49BE00C94CB2FCF93DF93E0E5FBE0CCE4DBE00C
:20588000A8E4BBE0919189918095892B8D938BE0E435F807B9F7DF91CF9108951F93CF9308
:2058A000DF93EB0140918E0250E0292F30E04217530709F066C090918F02981362C010919F
:2058C000990211FF3BC010927A028CE280937B020E94CA2A82E18093990260E081E090E04E
:2058E0000E94772A109290021092910280913C0180939202109293028D5F80933C0182E032
:205900008093A00284E08093A10285E08093A2021092A30290E69093980280939A0288E704
:2059200080939B0222E040E250E06AE182E30E940F2A8AE390E00E94D72723C014FF21C084
:205940000E94832B9093620B8093610B892B91F02091980230E044E0359527954A95E1F7F7
:20596000220F331F220F331F2E5D3F4FC217D30758F407C010FF05C060E080E090E00E94BC
:20598000DC2A80E090E001C0C901DF91CF911F910895EF92FF920F931F93CF93DF931F929E
:2059A000CDB7DEB77C018091370B882319F0C7010E944A24E114F10409F0BDC08091630B93
:2059C000857051F08091340B9091350B892B21F40E94BF278111C7C08091340B9091350BC5
:2059E00001969093350B8093340B80917C0B813009F07CC08091630B81FF78C082E0809331
:205A00007C0B80913D018F5F80933D0110917A0B00917B0B8F71F82E80917D0B20E2829F52
:205A2000C0011124F82A88E39BE00E94642B68E37BE0882319F08EE69BE002C084E69BE047
:205A40000E94002BE8E0EE2EE09276021092770249E050E068E67BE088E792E00E946F3765
:205A60008CE280937B0286E0809381020E94652A00938E0210938F028BE080938C02F09216
:205A80008D02E0E9F2E0DF011D92EA94E9F780913C01809392028D5F80933C0180E6809345
:205AA000980282E08093990293E090939A0210929B0210929C0210929D0210929E02109266
:205AC0009F028093A00294E09093A1028093A20286E28093A30222E040E250E06AE182E35B
:205AE0000E940F2A8AE390E00E94D7278CE39BE00E94642B882341F080916C0B811104C079
:205B000080916D0B8823C9F188E39BE00E94642B882309F4D4C180916A0B8111D0C1809189
:205B20006B0B8111CCC188E39BE00E94192B81E080936B0BC4C1B9E2EB16F10408F4BFC188
:205B400010917602183009F5809177028630E9F444E050E060E57BE080E992E00E9487379A
:205B6000892B99F445C084E49BE00E94192B8091630B88608093630B2FCF8CE39BE00E94A4
:205B8000192B81E080936D0BBFCFFAE2EF16F10408F495C1183009F092C18091770281116F
:205BA0008EC180917802853409F089C144E050E060E57BE088E892E00E948737892B09F428
:205BC00081C044E050E068E47BE088E892E00E948737892B09F476C044E050E06CE272E06C
:205BE00088E892E00E948737892B09F068C16AC080917F02813029F580E792E00E94BF2A9E
:205C000010927E0282E080937F0260E872E08AE892E00E94D62F64E57BE080E892E00E9427
:205C2000D62F66E872E080E992E00E94CB2F60E57BE086E892E00E94CB2F8AE290E00E94AE
:205C4000D7278091630B83FF0CC010917F02123041F464E67BE084E49BE00E944D2B8111AC
:205C600028C080916C0B81110CC080916D0B882341F06EE67BE08CE39BE00E944D2B8111AC
:205C80001BC080916A0B81111AC180916B0B882309F415C16EE67BE088E39BE00E944D2B82
:205CA000882309F40CC181E080936A0B10926B0B06C11093630BD5CF81E080936C0B109265
:205CC0006D0BDFCF80918102813009F580918C028830E9F4E091740BF091750B309719F066
:205CE00084E892E009950E94CA2A10928C0290918E02983F28F080918F028F5F80938F028E
:205D0000985F90938E02C7010E94D727D8C00E94692F811105C0E6E3EE16F10430F4CFC0D3
:205D2000809181028131B9F7C4C080918102863009F0C5C080918E028B3009F0ACC044E03C
:205D400050E068E37BE084E892E00E948737892B09F0B5C02091990222FF13C0E091780BD9
:205D6000F091790B309759F080918F0220E030E040E050E063E0829586958770099585E09D
:205D800078C029830E94832B8C0180917C0B2981823071F5822F807122712231E9F460E043
:205DA00080E090E00E94DC2A88E180939902E091760BF091770B309739F080918D028295B8
:205DC00086958770099502C080E090E023E020937C0B0E94A32A73C091E090937C0B8111F5
:205DE00003C0C801019602C080E090E064E039C0833009F041C00115110509F43FC0E0916B
:205E0000780BF091790B3097C9F14091980250E064E0559547956A95E1F7440F551F440FE3
:205E2000551FC70108974E5D5F4F8417950708F4AC01C801840F951FE816F90620F4970195
:205E4000241B350B01C0980180918F0260E082958695877009958091360B882329F068E062
:205E6000C8010E94DC2A2BC069E0C8010E94DC2A86E080937C0B23C0853009F120FF06C095
:205E80008330E9F069E0C8010196F0CF01151105B1F060E0E5CFB70180913A0190913B01EC
:205EA0000F90DF91CF911F910F91FF90EF900C944E2CC7010E94702F882309F42CCF80E0EF
:205EC00090E00F90DF91CF911F910F91FF90EF90089581E090917E0B911101C080E008957D
:205EE000AF92BF92CF92DF92EF92FF920F931F93CF93DF93CFE7DBE073E8C72E7BE0D72EE3
:205F0000E12CF12C40E020917E0B30E0E216F306B4F55A819B8120918E0230E0A92EB12C57
:205F20002A153B0521F580918F02851320C0F60120812223E1F00091910210E0085011097E
:205F40002091900230E0322F2227020F131F40918C0250E0542F442720918D02422BE8816E
:205F6000F98124E932E064E872E0099541E0FFEFEF1AFF0A259685E0C80ED11CC4CF842F02
:205F8000DF91CF911F910F91FF90EF90DF90CF90BF90AF900895FB01408151816281738174
:205FA000FC014083518362837383089526E0FB01DC0101900D922A95E1F70895CF93DF93BE
:205FC000F90150E0EC01A881BA2FBF7D01F1AA30F1F0511116C0B081AB1310C0A181AA23C9
:205FE00011F031960CC0DC01119651E0EC0189818D3309F050E0F901CD0101C0F90101965E
:20600000E1CFDC01FB0150E0415051090EC05130C1F380E011C09A3071F0963261F0282F0D
:2060200030E0241735073CF491938E2F861B9D91292F2F7D81F71082DF91CF910895EF92FD
:20604000FF920F931F93DC01ED91FC9111971A960D911C911B9718962D913C9119970684AB
:20606000F785E02D7B0140E050E060E070E009951F910F91FF90EF9008958EBD0DB407FE91
:20608000FDCF08952CB5982F93702C7F922B9CBD9DB582FB882780F99E7F982B9DBD08955D
:2060A000EF92FF920F931F93CF93DF931F92CDB7DEB77C01062F142F40E451E060EF70E0F3
:2060C00029830E940C2386E392E0F7019183808300A311A3298124A3178A0F90DF91CF9181
:2060E0001F910F91FF90EF900895CF93DF93EC01862FEE8DFF8D208198A59095922390835D
:20610000EC8DFD8D20819FA19095922390830E943D30EC8DFD8D80819FA1892B8083DF9134
:20612000CF910895662311F061E201C060E20C947530CF93DF93EC01862FEE8DFF8D9081BF
:2061400028A5922B9083EC8DFD8D20819FA19095922390830E943D30EC8DFD8D80819FA17E
:20616000892B8083DF91CF9108950F931F93CF93DF931F92CDB7DEB78C01872FD8015E96F9
:20618000ED91FC915F97908198962C919897922B90835C96ED91FC915D97208197969C9117
:2061A00090959223908369830E943D306981862F0E943D30D8015C96ED91FC915D9780817E
:2061C00097969C91892B80830F90DF91CF911F910F910895CF93DF93EC0161E089A10E9484
:2061E000880A61E088A10E94880A48A150E0FA01EC5DFC4FE491F0E0EE0FFF1FEC5BFC4FD5
:20620000859194919D8F8C8F29A130E0F901EC5DFC4F849190E0880F991F8C5B9C4FFC01F1
:20622000859194919F8F8E8FFA01EC5FFC4F44914FA3F901EC5FFC4F249128A70E94D01FDB
:2062400080E00E9442308CB58F7D8CBD8CB5837F8CBDEC8DFD8D90818FA1809589238083A0
:2062600081E08F8B8CA1882319F161E00E94880A61E08CA10E94C10A64EF71E080E090E0FD
:206280000E94E90960E08CA10E94C10A64EF71E080E090E00E94E90961E08CA10E94C10AAD
:2062A00064EF71E080E090E0DF91CF910C94E909DF91CF910895CF93DF93EC016FEE0E94DB
:2062C000753063E0CE010E94993060E8CE010E94993062E0CE010E9499306FECCE010E94D2
:2062E000753060E0CE010E94993061ECCE010E94993060E3CE010E9499306DEECE010E94AF
:20630000753064E6CE010E94993063E0CE010E94993062E1CE010E94993061E8CE010E94A0
:20632000993068EECE010E94753065E8CE010E94993060E0CE010E94993068E7CE010E9467
:2063400099306BECCE010E94753069E3CE010E9499306CE2CE010E94993060E0CE010E9448
:20636000993064E3CE010E94993062E0CE010E94993067EFCE010E94753060E2CE010E9438
:2063800099306AEECE010E94753060E0CE010E94993060E0CE010E94993060ECCE010E9415
:2063A000753063E2CE010E94993061ECCE010E94753060E1CE010E94993065ECCE010E9419
:2063C00075306EE3CE010E94993068E2CE010E94993067ECCE010E94753066E8CE010E94E1
:2063E000993066E3CE010E94753068E4CE010E9499306AE3CE010E94753065E5CE010E94D1
:20640000993061EBCE010E94753060E0CE010E94993068E1CE010E94993066EBCE010E9492
:20642000753068E0CE010E94993062E8CE010E94993067E2CE010E94993062EFCE010E946C
:20644000753060E0CE010E94993066E2CE010E94753061E0CE010E94993060EECE010E9485
:2064600075306FE0CE010E94993061E3CE010E9499306BE2CE010E9499306CE0CE010E942C
:2064800099306EE0CE010E94993068E0CE010E9499306EE4CE010E94993061EFCE010E94DC
:2064A000993067E3CE010E94993067E0CE010E94993060E1CE010E94993063E0CE010E94DF
:2064C00099306EE0CE010E94993069E0CE010E94993060E0CE010E94993061EECE010E94AE
:2064E000753060E0CE010E9499306EE0CE010E94993064E1CE010E94993063E0CE010E94C2
:20650000993061E1CE010E94993067E0CE010E94993061E3CE010E94993061ECCE010E9479
:20652000993068E4CE010E94993068E0CE010E9499306FE0CE010E9499306CE0CE010E9444
:20654000993061E3CE010E94993066E3CE010E9499306FE0CE010E94993061E1CE010E9435
:20656000753068E770E080E090E00E94E90969E2CE01DF91CF910C947530CF93DF93EC0183
:206580000E94EA308F89882329F0CE01DF91CF910C945B31DF91CF910895AF92BF92CF9238
:2065A000DF92EF92FF920F931F93CF93DF93EC017B016A0159016AE20E947530B701CE01E8
:2065C0000E94B530B501CE010E94B5306BE2CE010E947530B601CE010E94B530B801CE0130
:2065E0000E94B5306CE2CE01DF91CF911F910F91FF90EF90DF90CF90BF90AF900C94753028
:20660000EF92FF920F931F93CF93DF93EC0179018885998568177907E4F48A859B85481749
:206620005907BCF477FD15C057FD13C08A010F5F1F4F9B012F5F3F4FCE010E94CD32B70193
:20664000CE01DF91CF911F910F91FF90EF900C94B530DF91CF911F910F91FF90EF900895ED
:20666000CF92DF92EF92FF920F931F93CF93DF93EC0179016801888599856817790714F50B
:206680008A859B8548175907ECF49A012E0D3F1D821793071CF47C01E41AF50A8A010E0D97
:2066A0001F1D015011099B01CE010E94CD32E114F10441F0B601CE010E94B53081E0E81A9C
:2066C000F108F5CFDF91CF911F910F91FF90EF90DF90CF900895CF92DF92EF92FF920F93DE
:2066E0001F93CF93DF93EC0179016801888599856817790714F52A853B8542175307ECF40F
:206700009B012E0D3F1D821793071CF47C01E61AF70A9B012E0D3F1D215031098A01CE014D
:206720000E94CD32E114F10441F0B601CE010E94B53081E0E81AF108F5CFDF91CF911F91F0
:206740000F91FF90EF90DF90CF900895AF92BF92CF92DF92EF92FF920F931F93CF93DF9382
:20676000EC01690158012885398562177307B4F58A859B85481759078CF5FB01EC0DFD1DE4
:206780002E173F071CF46901C61AD70A9A012A0D3B1D821793071CF45C01A41AB50A8A0161
:2067A0000A0D1B1D015011099B012C0D3D1D21503109CE010E94CD321A141B047CF4860191
:2067C000101611063CF4B701CE010E94B53001501109F6CF81E0A81AB108EECFDF91CF91A5
:2067E0001F910F91FF90EF90DF90CF90BF90AF9008951F93CF93DF93EC0163706D8B623072
:20680000C1F0633001F1613051F080EF90E09987888780E491E09B878A8718E41DC080E41D
:2068200091E09987888780EF90E09B878A8718E213C080EF90E09987888780E491E09B87D4
:206840008A8718E809C080E491E09987888780EF90E09B878A8718EE66E3CE010E947530E3
:20686000612FCE01DF91CF911F910C94993008950E9449371F920F920FB60F9211240BB663
:206880000F922F938F939F93EF93FF93E091B70BF091B80B8081E091BD0BF091BE0B82FDB3
:2068A00012C090818091C00B8F5F8F732091C10B821751F0E091C00BF0E0E955F44F958F21
:2068C0008093C00B01C08081FF91EF919F918F912F910F900BBE0F900FBE0F901F90189529
:2068E0001F920F920FB60F9211240BB60F922F933F934F935F936F937F938F939F93AF9337
:20690000BF93EF93FF9387EA9BE00E943335FF91EF91BF91AF919F918F917F916F915F912B
:206920004F913F912F910F900BBE0F900FBE0F901F90189587EA9BE00E94E73421E0892BBA
:2069400009F420E0822F08951092AA0B1092A90B88EE93E0A0E0B0E08093AB0B9093AC0BA3
:20696000A093AD0BB093AE0B82E592E09093A80B8093A70B85EC90E09093B40B8093B30B28
:2069800084EC90E09093B60B8093B50B80EC90E09093B80B8093B70B81EC90E09093BA0B04
:2069A0008093B90B82EC90E09093BC0B8093BB0B86EC90E09093BE0B8093BD0B1092C00B49
:2069C0001092C10B1092C20B1092C30B0895FC01818D228D90E0805C9F4F821B91098F73A0
:2069E00099270895FC01918D828D981731F0828DE80FF11D858D90E008958FEF9FEF089564
:206A0000FC01918D828D981761F0828DDF01A80FB11D5D968C91928D9F5F9F73928F90E008
:206A200008958FEF9FEF08958AE994E3892B41F080E090E0892B21F00E949A3481110DC0DD
:206A400080E090E0892B71F080E090E0892B51F00E940000811104C008950E940000F0CF96
:206A60000C9400000895FC01848DDF01A80FB11DA35ABF4F2C91848D90E001968F739927C4
:206A8000848FA689B7892C93A089B1898C9180648C93938D848D981306C00288F389E02D7D
:206AA00080818F7D80830895CF93DF93EC01888D8823C9F0EA89FB89808185FD05C0A8897F
:206AC000B9898C9186FD0FC00FB607FCF5CF808185FFF2CFA889B9898C9185FFEDCFCE0194
:206AE0000E943335E7CFDF91CF910895CF92DF92FF920F931F93CF93DF931F92CDB7DEB714
:206B00006C0181E0D60158968C9358975B969C915B975C968C915C97981307C05096ED91EC
:206B2000FC915197808185FD2EC0F601038D10E00F5F1F4F0F731127F02EF601848DF81232
:206B400011C00FB607FCF9CFD6015096ED91FC915197808185FFF1CFC60169830E94333522
:206B60006981EBCF838DE80FF11DE35AFF4F6083D6015B960C935B975296ED91FC915397B8
:206B8000808180620CC0D6015696ED91FC91579760835096ED91FC915197808180648083E6
:206BA00081E090E00F90DF91CF911F910F91FF90DF90CF9008954F925F926F927F92AF9226
:206BC000BF92CF92DF92EF92FF920F931F93CF93DF93CDB7DEB729013A01621B730B840B50
:206BE000950B29893A894B895C892A193B094C095D09298B3A8B4B8B5C8B9B01AC01698914
:206C00007A898B899C890E940638E418F50806091709A80197010E9458382A0D3B1D4C1DC5
:206C20005D1DCA01B901DF91CF911F910F91FF90EF90DF90CF90BF90AF907F906F905F90CE
:206C40004F900895CF93DF938230910510F482E090E0E091460CF091470C20E030E0A0E09F
:206C6000B0E0309739F14081518148175907B8F04817590771F482819381109729F01396F5
:206C80009C938E9312972CC09093470C8093460C27C02115310531F04217530718F0A9015B
:206CA000DB0101C0EF019A01BD01DF010280F381E02DD7CF21153105F9F0281B390B243035
:206CC000310580F48A819B816115710521F0FB019383828304C09093470C8093460CFE0131
:206CE000329644C0FE01E20FF31F8193919322503109398328833AC02091440C3091450C6E
:206D0000232B41F420910201309103013093450C2093440C2091000130910101211531057F
:206D200041F42DB73EB74091040150910501241B350BE091440CF091450CE217F307A0F4EF
:206D40002E1B3F0B2817390778F0AC014E5F5F4F2417350748F04E0F5F1F5093450C409320
:206D6000440C8193919302C0E0E0F0E0CF01DF91CF910895CF93DF93009709F487C0FC0150
:206D8000329713821282C091460CD091470C209781F420813181280F391F8091440C90911A
:206DA000450C8217930779F5F093450CE093440C6DC0DE0120E030E0AE17BF0750F41296B7
:206DC0004D915C9113979D014115510509F1DA01F3CFB383A28340815181840F951F8A1787
:206DE0009B0771F48D919C911197840F951F02969183808312968D919C91139793838283EB
:206E00002115310529F4F093470CE093460C3EC0D9011396FC93EE9312974D915D91A40F95
:206E2000B51FEA17FB0779F480819181840F951F0296D90111969C938E938281938113968B
:206E40009C938E931297E0E0F0E08A819B81009719F0FE01EC01F9CFCE0102962881398164
:206E6000820F931F2091440C3091450C2817390769F4309729F41092470C1092460C02C051
:206E800013821282D093450CC093440CDF91CF91089581E090E0F8940C949B38FC01882789
:206EA0009927E89421912032E9F3293010F02E30C8F32B3241F02D3239F4689404C00E94C8
:206EC000C437820F911D219120532A30C0F31EF4909581959F4F0895F8940C949B38FB0173
:206EE000DC0102C005900D9241505040D8F70895FB01DC014150504048F005900D920020AC
:206F0000C9F701C01D9241505040E0F70895FB01DC0104C08D910190801921F44150504091
:206F2000C8F7881B990B0895FC018191861721F08823D9F7992708953197CF010895FB01E8
:206F4000DC0101900D920020E1F70895FB01DC014150504048F001900D920020C9F701C08C
:206F60001D9241505040E0F70895BB272A3051F4992342F4BDE290958095709561957F4FB8
:206F80008F4F9F4F0C94CD377AE0979F902D879F802D910D11240895BB27FA01A62F6217C6
:206FA000710581059105330B30FB66F0AA27660F771F881F991FAA1FA21710F0A21B63950E
:206FC0003850A9F7A05DAA3308F0A95DA19336F7B111B1931082CA010C94F637F999FECFC1
:206FE00092BD81BDF89A992780B50895DC01FC01672F71917723E1F7329704C07C916D9362
:2070000070836291AE17BF07C8F30895DB018F939F930E947D38BF91AF91A29F800D911D14
:20702000A39F900DB29F900D11240895991B79E004C0991F961708F0961B881F7A95C9F75C
:2070400080950895AA1BBB1B51E107C0AA1FBB1FA617B70710F0A61BB70B881F991F5A95FB
:20706000A9F780959095BC01CD010895A1E21A2EAA1BBB1BFD010DC0AA1FBB1FEE1FFF1F0F
:20708000A217B307E407F50720F0A21BB30BE40BF50B661F771F881F991F1A9469F760959F
:2070A0007095809590959B01AC01BD01CF010895052E97FB1EF400940E946F3857FD07D03E
:2070C0000E94363807FC03D04EF40C946F3850954095309521953F4F4F4F5F4F0895909570
:2070E0008095709561957F4F8F4F9F4F0895EE0FFF1F0590F491E02D09940E948C38A59FC0
:20710000900DB49F900DA49F800D911D112408950790F691E02D0994A29FB001B39FC001C5
:20712000A39F700D811D1124911DB29F700D811D1124911D0895F894FFCF0000480C8000F5
:20714000010000007469692D3031FFFFFFFF63825363350141726475696E6F2D303000002E
:20716000000000000000000000000000000000000000000050000A010A496E697469616CE0
:20718000697A696E6720534420636172642E2E2E2020005B4552524F525D005B4F4B5D00FF
:2071A000496E697469616C697A696E672045746865726E65742E2E2E20002020444843507C
:2071C000206661696C656400202049503A20000A202047573A20000A2020444E533A20002C
:2071E000434845434B4544006331006332002A2A204C6F76652053696C766961202A2A0079
:207200006572726F72206F70656E696E6720746573742E7478740000000000F205070B0DB0
:207220000A006E616E00696E66006F7666002E0000000000D10BE70BC20C210C2B0C020C43
:207240002F00000000001C19070B00000000E521070B383406200C212321BD2039216E21D7
:207260008C213D228D21FFFFFFFFFFFF00000000E521070B0033062030336B33BD20A63332
:207280001F3092303D228D21000000007635070BE7340035F2345435FFFFFFFFFFFFFFFF1C
:2072A000FFFFFFFFFFFFFFFFFFFFFFFFFFFFFFFFFFFFFFFFFFFFFFFFFFFFFFFFFFFFFFFFEE
:2072C000FFFFFFFFFFFFFFFFFFFFFFFFFFFFFFFFFFFFFFFFFFFFFFFFFFFFFFFFFFFFFFFFCE
:2072E000FFFFFFFFFFFFFFFFFFFFFFFFFFFFFFFFFFFFFFFFFFFFFFFFFFFFFFFFFFFFFFFFAE
:20730000FFFFFFFFFFFFFFFFFFFFFFFFFFFFFFFFFFFFFFFFFFFFFFFFFFFFFFFFFFFFFFFF8D
:020000040001F9
:20FC00000F92CDB7DEB7112484B714BE81FFF1D085E08093810082E08093C00088E18093FD
:20FC2000C10086E08093C20080E18093C4008EE0CAD0209A26E080E39CEF31E09093850021
:20FC40008093840036BBB09BFECF189AA8952150A9F700E010E0EE24E394E1E1DE2EF3E00A
:20FC6000FF2EA5D0813471F4A2D08983B2D08981823809F48BC0813811F484E001C083E076
:20FC80008FD08BC0823411F484E103C0853419F485E0A7D082C0853591F489D0A82EBB24A6
:20FCA00086D0082F10E0102F00270A291B29812F881F8827881F8BBF000F111F6DC08635CC
:20FCC00021F484E08ED080E0DBCF843609F040C06ED06DD0C82E6BD080EE0030180718F41B
:20FCE000F801F7BEE895A12C51E0B52E60D0F50181935F01CE16D1F7F0EE00301F0718F076
:20FD0000F801F7BEE89565D007B600FCFDCFF801A0E0B1E02C9130E011968C91119790E04B
:20FD2000982F8827822B932B12960C01E7BEE8951124329682E0A030B80761F785E0F80167
:20FD400087BFE89507B600FCFDCFD7BEE89525C08437A9F42CD02BD0B82E29D03AD0CB2C35
:20FD60004801F40186911CD00894811C911CCA94C1F70F5F1F4FBA940B0D111D0EC085374C
:20FD800039F427D08EE10CD087E90AD085E078CF813511F488E017D01CD080E101D061CFA6
:20FDA0009091C00095FFFCCF8093C60008958091C00087FFFCCF8091C00084FD01C0A8951B
:20FDC0008091C6000895E0E6F0E098E1908380830895EDDF803219F088E0F5DFFFCF84E1F7
:1CFDE000DFCFCF93C82FE3DFC150E9F7F2DFCF91089580E0E8DFEE27FF27099480
:00000001FF
